:020000040800F2
:10000000600600206D0100087501000877010008F6
:10001000790100087B0100087D0100080000000054
:100020000000000000000000000000007F01000848
:10003000810100080000000083010008850100081C
:100040008701000887010008870100088701000870
:100050008701000887010008870100088701000860
:100060008701000887010008870100088701000850
:100070008701000887010008870100088701000840
:100080008701000887010008870100088701000830
:100090008701000887010008870100088701000820
:1000A0008701000887010008870100088701000810
:1000B0008701000887010008000000008701000890
:1000C0008701000800000000000000008701000810
:1000D0000000000087010008870100080000000000
:1000E00087010008870100088701000800F002F876
:1000F00000F02CF80AA090E8000C82448344AAF196
:100100000107DA4501D100F021F8AFF2090EBAE893
:100110000F0013F0010F18BFFB1A43F0010318473B
:1001200030030000400300000023002400250026C7
:10013000103A28BF78C1FBD8520728BF30C148BF4A
:100140000B6070471FB51FBD10B510BD00F048F91A
:100150001146FFF7F7FF00F02AF800F066F903B444
:10016000FFF7F2FF03BC00F06BF90000094880477D
:1001700009480047FEE7FEE7FEE7FEE7FEE7FEE789
:10018000FEE7FEE7FEE7FEE704480549054A064BA1
:1001900070470000AD010008ED000008600000207D
:1001A00060060020600200206002002070471A48AC
:1001B000806940F0040018498861042017490860EC
:1001C00000F0B5F800F0A9F825E014480830006800
:1001D00010F0010F11D01E2000F0F6F802210020CF
:1001E00000F08DF80EA000F0DBF80721012000F0F0
:1001F00086F80DA000F0D4F80DE00221002000F0F8
:100200007EF807A000F0CCF80721012000F077F875
:1002100006A000F0C5F8D8E7001002400008014031
:1002200053776974636800004F4E20004F464600C4
:100230000022002104E000E0521C3C2AFCDB491CA7
:100240008142F8DB704700B55C48006820F002008E
:100250005A490860DC20FFF7EBFF5848006840F07F
:10026000020056490860DC20FFF7E2FF53480068AF
:1002700020F0020051490860DC20FFF7D9FF00BDE3
:1002800030B504460D464D48006820F0F3004B4958
:1002900008600846006804F0F00108434749086018
:1002A000012D05D10846006840F00100086005E016
:1002B0004248006820F0010040490860FFF7C3FF92
:1002C0003E48006820F0F3003C490860084600689A
:1002D00004F00F0140EA011038490860012D05D1F2
:1002E0000846006840F00100086005E033480068F7
:1002F00020F0010031490860FFF7A5FF30BD70B55F
:1003000005460E460DB9002400E04024344344F075
:1003100080000021FFF7B4FF70BD00B5002101206F
:10032000FFF7AEFF00210220FFF7AAFF00BD00B5D6
:100330002348806940F008002149886121481F490D
:100340000C3908601D48006820F0F3001B49086064
:100350004FF4FA40FFF76CFF4FF4FA40FFF768FFE5
:100360004FF4FA40FFF764FF1448006820F00100E2
:10037000124908600846006820F00200086020204A
:100380000860FFF760FF00212820FFF779FF0021B8
:100390000E20FFF775FF00210620FFF771FF00BD5B
:1003A00030B505462C4604E020780121FFF768FFB0
:1003B000641C14B120780028F6D130BD0C0C01402B
:1003C000001002403300333300EB80035A00002159
:1003D00000E0491C9142FCDB704770477047704752
:1003E000754600F029F8AE4605006946534620F0F0
:1003F0000700854618B020B5FFF7C6FEBDE82040CF
:100400004FF000064FF000074FF000084FF0000BD0
:1004100021F00701AC46ACE8C009ACE8C009ACE883
:10042000C009ACE8C0098D4670470446AFF30080B0
:100430002046FFF794FE00000048704700000020AF
:1004400001491820ABBEFEE72600020070470000FD
:100450006004000800000020600600002801000879
:040000050800016D81
:00000001FF
